:101800003BC06FC054C053C052C051C050C04FC045
:101810004EC04DC04CC04BC04AC049C048C047C074
:1018200046C045C044C0040309041C037700770088
:1018300077002E00660069007300630068006C008A
:101840002E00640065000E03550053004200610045
:101850007300700012011001FF000008C016DC05C3
:101860000201010200010902120001010080320997
:10187000040000000000000011241FBECFE5D4E0EA
:10188000DEBFCDBF10E0A0E6B0E0E6E6FFE102C0BB
:1018900005900D92A636B107D9F710E0A6E6B0E0A4
:1018A00001C01D92AC39B107E1F770D15AC3A8CF7E
:1018B000A82FB92F80E090E041E050EA609530E039
:1018C00009C02D9182279795879510F08427952739
:1018D000305EC8F36F5FA8F30895EADF8D939D93A0
:1018E0000895CF93CFB7CF93C395849BE9F7849B9B
:1018F0000BC0849B09C0849B07C0849B05C0849B4C
:1019000003C0849B01C0C0C0C0917F00DF93DD276E
:10191000CA57DF4F2F932FEF849B03C02F91DF9186
:10192000E6CF0F931F934F936F9300B304FB20F9FF
:101930003F933BE05F931EC04E7F012F10B31471A5
:10194000E1F0216000001DC0102F4D7F22600000DB
:1019500000B3047191F01DC04B7F2460012F000083
:1019600010B3147151F01EC010B3147131F0477FE1
:1019700028601BC010B3147109F462C04FEF297FB7
:10198000D9F2012704FB21F900B30471B1F3237FDD
:10199000D9F2102714FB22F900C010B3147169F3B7
:1019A000277ED1F2012704FB23F92F7CE9F200B353
:1019B000047119F3102714FB24F92F7929F100C0C1
:1019C00010B31471E9F1012704FB25F92F7311F10C
:1019D00000C000B30471A1F1102714FB26F92230D6
:1019E000F8F000C010B3147159F1012704FB27F976
:1019F0002430E0F04227000000B34993102714FB85
:101A000020F93150C8F0B6CF4F7E00B30471C1F059
:101A10002061D3CF206210B3147191F04F7DD6CFE7
:101A20004F7B00B3047161F02064D9CF4F7710B3BE
:101A3000147131F02068DCCF10E41ABF002717C002
:101A40003B503195C31BD04010E41ABF0881033CC2
:101A5000F9F00B34E9F020917D001981110F121378
:101A6000EDCF093651F10D3211F0013E39F70093F7
:101A700084005F913F916F914F911F910F912F9132
:101A8000DF91CAB7C6FD30CFCF91CFBFCF911895A8
:101A900020918400222369F310918200112331F5F3
:101AA000343032F13093820020937E0010917F0019
:101AB0003BE0311B30937F001BC00091820001305E
:101AC000ACF40AE53091600034FD13C0009360006F
:101AD000C2E7D0E012C005271127000019C0052772
:101AE00011271FC005271127000024C04AE502C0A6
:101AF00032ED432FC4E1D0E032E011B31461949A87
:101B000002B311BB54E120E866E020FF05272795CA
:101B100002BB17951C3FF8F66A95B9F720FF052719
:101B20002795000002BB17951C3FC8F620FF05272C
:101B30002795179566E01C3F02BBA0F629913A95C0
:101B400021F70B7E10918300110F02BBC651D040CC
:101B500011F010937D0010E41ABF006111B31B7ED9
:101B6000402F4B7E53E05A95F1F700C002BB11BBEA
:101B700042BB7FCF12BAF8941BBE15BE81E08BBF6B
:101B80001BBEE0917000F0917100099588E10FB6DD
:101B9000F89481BD11BC0FBE979A04B601FECBC16B
:101BA00014BE81E08BBF82E08BBF8799C4C185B72B
:101BB000826085BF8BB780648BBF8C9A20E005C0A4
:101BC000A89586EA9EE00197F1F72150C9F78C9815
:101BD0007894FF2400E090918200935097FD2EC1ED
:101BE00080917F00CCE0D0E0C81BD109CA57DF4FFD
:101BF00080917E008D3209F0C4C0983009F01CC17C
:101C000083EC809372008AE58093600010926A00F2
:101C10003881832F80762981882309F443C086E6A2
:101C200090E090938100809380002330C9F49B81E1
:101C30008C812A81203339F48370E82FF0E0EE594B
:101C4000FF4F808109C0203A11F476D105C0203CB5
:101C500011F46D8179D180E08093690094E087C0B0
:101C6000253011F491E083C0822F8450863098F49F
:101C70008A819B8190936D0080936C00293081F064
:101C80009E8190936E008D81827080936F0037FDEE
:101C900069C02FEF68C0223019F481E080936B0097
:101CA00090E065C08A8110927B00222331F410926B
:101CB0007C002BE730E092E050C0253019F480938F
:101CC000830048C02630B1F58B81813019F484E55A
:101CD00098E104C0823041F486E698E19093810057
:101CE0008093800092E122C08330F9F48A818823B6
:101CF00041F486E298E1909381008093800094E023
:101D000015C0813041F48AE298E19093810080937C
:101D100080009CE10BC0823041F486E498E190930E
:101D20008100809380009EE001C090E080E4809379
:101D30006A001DC0283019F425E830E009C02930B8
:101D400019F48093850006C02A3021F42BE730E097
:101D500091E003C02BE730E090E0309381002093C6
:101D6000800005C0292F80E880936A0007C08F811A
:101D7000882319F42E81291708F0292F2093610058
:101D80005BC080916A0087FF57C080916E00592F19
:101D9000891708F4582F851B80936E0060E0882314
:101DA00009F461E070916F00E0916C00F0916D00BA
:101DB00040E037C0CF018F739070892B49F4F894BD
:101DC00083E080935700E895789407B600FCFDCF38
:101DD0004E5FF8948991999121E00C01209357006E
:101DE000E895112478949F012E5F3F4FC9018F73AE
:101DF0009070892B31F0662399F0451788F077238E
:101E000079F0F89485E080935700E895789407B6C8
:101E100000FCFDCFF89481E180935700E895789419
:101E2000F901451708F4C6CFF0936D00E0936C00FC
:101E3000662311F010926100109282008091600080
:101E400084FF65C0809161008F3F09F460C0182F46
:101E5000893008F018E0811B809361008091720046
:101E600098E8892780937200112309F43EC080917D
:101E70006A0087FF1EC080916E00811708F4182F3A
:101E8000811B80936E00E0916C00F0916D00A3E7E0
:101E9000B0E003C084918D933196812F90E08D58EE
:101EA0009F4FA817B907B1F7F0936D00E0936C004E
:101EB0001AC0E0918000F091810086FF09C0912F47
:101EC000A3E7B0E084918D9331969150D9F707C084
:101ED000912FA3E7B0E081918D939150E1F7F093BA
:101EE0008100E0938000193060F483E790E0612F77
:101EF000F4DC612F6C5F6C3041F08FEF80936100F8
:101F000004C08FEF809361006EE16093600094E104
:101F100080B3847131F49150D9F7109283001092FC
:101F20007D0080916B00882321F0FA9411F4015018
:101F300011F0879B50CE1EDEE199FECF9FBB8EBB7A
:101F4000E09A99278DB30895262FE199FECF9FBB84
:101F50008EBB2DBB0FB6F894E29AE19A0FBE0196A4
:061F60000895F894FFCF84
:061F66005AFF1E93070064
:0400000300001800E1
:00000001FF
